:0200000480007A
:100000006F00C004732F2034930F8000630AFF0336
:10001000930F90006306FF03930FB0006302FF038A
:10002000170F0080130F0FFE63040F0067000F000F
:10003000732F203463540F006F00400093E19153FD
:10004000171F000023203FFC6FF09FFF732540F136
:1000500063100500970200009382020173905230F2
:10006000735000189702000093820202739052307E
:10007000B70200809382F2FF7390023B9302F0017B
:100080007390023A9702000093828201739052307B
:100090007350203073503030735040309301000063
:1000A00097020000938242F67390523013051000BD
:1000B0001315F501634C05000F00F00F93011000BC
:1000C0009308D0051305000073000000970200801C
:1000D000938242F3638E020073905210B7B2000015
:1000E000938292107390223073232030E39862F44D
:1000F00073500030970200009382420173901234D3
:10010000732540F17300203093012000930000001C
:100110001301100063962000631A302A6316300022
:10012000E39E20FE6314302A9301300093001000F8
:100130001301000063962000631A30286316300014
:10014000E39E20FE63143028930140009300F0FFEB
:100150001301100063962000631A302663163000E6
:10016000E39E20FE6314302693015000930010009C
:100170001301F0FF63962000631A302463163000E9
:10018000E39E20FE6314302493016000930000007E
:1001900013010000639420006314300063183022C0
:1001A000E39E20FE930170009300100013011000E5
:1001B0006394200063143000631A3020E39E20FE15
:1001C000930180009300F0FF1301F0FF639420007F
:1001D00063143000631C301EE39E20FE93019000E8
:1001E0001302000093000000130100006390201E22
:1001F0001302120093022000E31652FE9301A000A6
:10020000130200009300000013010000130000001F
:10021000639E201A1302120093022000E31452FE80
:100220009301B000130200009300000013010000CE
:100230001300000013000000639A2018130212003C
:1002400093022000E31252FE9301C000130200004B
:1002500093000000130000001301000063982016B3
:100260001302120093022000E31452FE9301D00007
:1002700013020000930000001300000013010000AF
:100280001300000063942014130212009302200054
:10029000E31252FE9301E0001302000093000000FD
:1002A00013000000130000001301000063902012EF
:1002B0001302120093022000E31252FE9301F00099
:1002C000130200009300000013010000639020104F
:1002D0001302120093022000E31652FE9301000164
:1002E000130200009300000013010000130000003F
:1002F000639E200C1302120093022000E31452FEAE
:10030000930110011302000093000000130100008C
:100310001300000013000000639A200A1302120069
:1003200093022000E31252FE930120011302000009
:1003300093000000130000001301000063982008E0
:100340001302120093022000E31452FE93013001C5
:1003500013020000930000001300000013010000CE
:100360001300000063942006130212009302200081
:10037000E31252FE930140011302000093000000BB
:10038000130000001300000013010000639020041C
:100390001302120093022000E31252FE9300100099
:1003A000639A0000938010009380100093801000E7
:1003B000938010009380100093801000930E300003
:1003C000930150016394D001631030020F00F00FCD
:1003D000638001009391110093E111009308D0050F
:1003E00013850100730000000F00F00F930110004F
:1003F0009308D0051305000073000000731000C0BF
:0404000000000000F8
:1010000000000000000000000000000000000000E0
:1010100000000000000000000000000000000000D0
:1010200000000000000000000000000000000000C0
:1010300000000000000000000000000000000000B0
:081040000000000000000000A8
:040000058000000077
:00000001FF
